:10000000831600308500860083125E2880309B00B6
:1000100080308606F0309A0056209B0B0828080096
:1000200090309B0080308606D5309A0056209B0B7E
:1000300012280800A0309B0080308606BD309A0050
:1000400056209B0B1C280800B0309B008030860691
:10005000B2309A0056209B0B26280800C0309B0027
:10006000803086069F309A0056209B0B302808006F
:10007000D0309B00803086068D309A0056209B0B36
:100080003A280800E0309B00803086067E309A00D7
:1000900056209B0B44280800F0309B0080308606D9
:1000A00077309A0056209B0B4E2808000000000075
:1000B0000000000000009A0B5628080006201A20B5
:1000C00024202E202E202E202E202E2006201A2006
:1000D00024202E202E202E202E202E2006201A20F6
:1000E00024202E202E201A201A20062006201A2036
:1000F0001A201020102010201020102056205620EA
:100100001A201020062006205620062006201A203D
:100110001A202E202E202E202420242024202420AB
:1001200024201A2024202E202E201A201A201020CD
:1001300010205620102010200620062006205620D1
:0401400006205E280F
:00000001FF
